:100000008A110A1205280000090083169F01831235
:10001000073099008B13831605108510051185157F
:100020000516851683122030BA000330BB006430F9
:10003000A000A1010E25051485140515C830A000E7
:10004000A1010E250510851005116430A000A10145
:100050000E25AB220F232924C830A000A1010E25B4
:10006000AF012F080A3C031C4A286D24B001300858
:10007000323C031C4428A3213230A000A1010E25EC
:100080000130B007031C37281F3083050130AF074C
:10009000031C31281F308305C830A000A1010E25A4
:1000A0008F24C830A000A1010E255D20C830A0001B
:1000B000A1010E258F242C285C280514F430A00003
:1000C0000130A1000E25AF012F081D3C031C9A2909
:1000D0003E08AD000130AE00A0242C08BD003D0854
:1000E000013C031D742859231F3083053D08023C41
:1000F000031D7B288E231F3083053D08033C031D11
:1001000082286A231F3083053D08043C031D89288B
:10011000A7231F3083053D08053C031D902891232C
:100120001F3083053D08063C031D9728A3231F307D
:1001300083053D08073C031D9E28A9231F30830526
:100140003D08083C031DA5288B231F3083053D086F
:10015000093C031DAC287A231F3083053D080A3C67
:10016000031DB328C5231F3083053D080B3C031D29
:10017000BA2886231F3083053D080C3C031DC12887
:1001800082231F3083053D080D3C031DC8289F2393
:100190001F3083053D080E3C031DCF2801241F306E
:1001A00083053D080F3C031DD628E3231F3083053C
:1001B0003D08103C031DDD289A231F3083053D08B0
:1001C000113C031DE428AD231F3083053D08123C7C
:1001D000031DEB2808241F3083053D08133C031D35
:1001E000F228D7231F3083053D08143C031DF9284E
:1001F000CB231F3083053D08153C031D0029B22386
:100200001F3083053D08163C031D072966231F3058
:1002100083053D08173C031D0E290F241F3083055D
:100220003D08183C031D1529FB231F3083053D089D
:10023000193C031D1C2961231F3083053D081A3C0E
:10024000031D232971231F3083053D081B3C031D1B
:100250002A295C231F3083053D081C3C031D3129DE
:1002600016241F3083053D081D3C031D3829DD235E
:100270001F3083053D081E3C031D3F29D1231F303D
:1002800083053D081F3C031D46297D231F30830540
:100290003D08203C031D4D2975231F3083053D0873
:1002A000213C031D5429E9231F3083053D08223CCE
:1002B000031D5B29F5231F3083053D08233C031DE7
:1002C0006229BB231F3083053D08243C031D692997
:1002D0006C231F3083053D08253C031D70299523A1
:1002E0001F3083053D08263C031D7729EF231F306F
:1002F00083053D08273C031D7E29B6231F30830557
:100300003D08283C031D8529C0231F3083053D0877
:10031000293C031D8C291C241F3083053D082A3CE1
:10032000031D932922241F30830552240130AF0777
:10033000031C64281F308305F430A0000130A100A5
:100340000E25051008008519A629B3211F30830545
:10035000051AAB29D8211F308305851AB0290E2232
:100360001F30830508003208A0003308A1000430C4
:10037000A3004C30F224031DC1299030B20001309B
:10038000B3001F3083053208643EB20033080318FF
:10039000013E003EB30005149630A000A1010E25D9
:1003A0008F2405100F23C830A000A1010E250800DE
:1003B0003408A0003508A100A3011E30EC24031D61
:1003C000E4295A30B400B5011F3083050F303402E0
:1003D000B4000030031C013E3502B5003408B600FD
:1003E0003508B7003408A6003508A7000330A2007E
:1003F000A301BA24B8002508B90005149630A0005E
:10040000A1010E259A2341249F234124AD230510E9
:100410000F23C830A000A1010E2508003C08083CAD
:10042000031D132ABC011F3083053C08013EBC009C
:1004300005149630A000A1010E253C08013C031DC7
:10044000222ACB231F3083053C08013C031D2A2AA6
:100450000430BE001F3083053C08023C031D312AD6
:10046000D1231F3083053C08023C031D392A093083
:10047000BE001F3083053C08033C031D402AD723E0
:100480001F3083053C08033C031D482A0E30BE0084
:100490001F3083053C08043C031D4F2ADD231F3019
:1004A00083053C08043C031D572A1230BE001F3050
:1004B00083053C08053C031D5E2AE3231F308305AA
:1004C0003C08053C031D662A1730BE001F3083051B
:1004D0003C08063C031D6D2AE9231F3083053C08B8
:1004E000063C031D752A1C30BE001F3083053C08E6
:1004F000073C031D7C2AEF231F3083053C08073C83
:10050000031D842A2030BE001F3083053C08083CB0
:10051000031D8B2AF5231F3083053C08083C031D6F
:10052000932A2530BE001F3083053C08093C031D7B
:100530009A2AFB231F3083053C08093C031DA22A8D
:100540002A30BE001F30830505100F23C830A000DD
:10055000A1010E2508008B13003083169B001C148C
:1005600000001A088312B10031086E3C0318B92A42
:10057000BF2A1F308305323031020318C12A4630AA
:10058000B1001F3083053108A600A7010A30A20080
:10059000A301BA24B2002508B300013083169B00E2
:1005A0001C1400001A088312B10031085A3C0318C9
:1005B000DA2AE02A1F3083050F3031020318E22ABD
:1005C0001E30B1001F3083053108B400B501310879
:1005D000B600B7013108A600A7010430A200A301AC
:1005E000BA24B8002508B900023083169B001C14F9
:1005F00000001A088312B1003108083C0318012BCF
:10060000072B1F308305023031020318092B0430F9
:10061000B1001F3083053108BC008B1708008B1315
:100620003208A0003308A1000A30A200A301D024A0
:10063000BF002108C0003F08B100003083169B00B6
:100640008312310883169A001C1555309D00AA307C
:100650009D009C149C182A2B1C1183128C133408A7
:10066000B100013083169B008312310883169A0073
:100670001C1555309D00AA309D009C149C183E2BE3
:100680001C1183128C133C08B100023083169B00AE
:100690008312310883169A001C1555309D00AA302C
:1006A0009D009C149C18522B1C1183128C138B17C9
:1006B00008006D247E2408007E246D246D246D24A2
:1006C00008007E246D247E246D2408007E246D2481
:1006D0006D2408006D2408006D246D247E246D2493
:1006E00008007E247E246D2408006D246D246D2472
:1006F0006D2408006D246D2408006D247E247E2462
:100700007E2408007E246D247E2408006D247E242F
:100710006D246D2408007E247E2408007E246D2430
:1007200008007E247E247E2408006D247E247E24FE
:100730006D2408007E247E246D247E2408006D2410
:100740007E246D2408006D246D246D2408007E2411
:1007500008006D246D247E2408006D246D246D2412
:100760007E2408006D247E247E2408007E246D24CF
:100770006D247E2408007E246D247E247E240800BF
:100780007E247E246D246D2408007E247E247E2415
:100790007E247E2408006D247E247E247E247E24F4
:1007A00008006D246D247E247E247E2408006D24A0
:1007B0006D246D247E247E2408006D246D246D2418
:1007C0006D247E2408006D246D246D246D246D2419
:1007D00008007E246D246D246D246D2408007E2481
:1007E0007E246D246D246D2408007E247E247E24C6
:1007F0006D246D2408007E247E247E247E246D24B6
:1008000008006D247E246D247E246D247E2408003F
:100810007E247E246D246D247E247E2408006D2495
:100820006D247E247E246D246D2408007E246D2496
:100830006D247E246D2408007E246D246D246D2497
:100840007E2408007E246D246D246D246D247E2476
:1008500008002C30A0000130A1000E259A2341246D
:100860009F234124AD2352242C30A0000130A1004D
:100870000E25080005113408A0003508A1000E253A
:10088000080005113408A0003508A1000E25340821
:10089000A0003508A1000E253408A0003508A100ED
:1008A0000E25080005113408A0003508A1000E250A
:1008B0003408A0003508A1000E253408A000350832
:1008C000A1000E253408A0003508A1000E2534082B
:1008D000A0003508A1000E2508000515053084008C
:1008E0000230AA003208A0003308A1003608A20096
:1008F0003708A300492505113A24080005150530DD
:1009000084000230AA003208A0003308A100380891
:10091000A2003908A300492505113A24080005154D
:10092000053084000230AA003208A0003308A1007C
:100930003A08A2003B08A300492505113A24080003
:100940008316811283120108A000A1012D08A200C4
:10095000A301D0242408BF002508C0003F082E07AB
:10096000BF0040080318013E003EC0003F08AC0035
:100970000800B92C1030A800A101A001A70CA60CFA
:10098000031CC82C2208A00723080318230FA10763
:10099000A10CA00CA50CA40CA80BBE2C24080800CC
:1009A0001030A600A501A401210DA40DA50D22085B
:1009B000A4022308031C230FA5020318E62C220817
:1009C000A40723080318230FA5070310A00DA10DEA
:1009D000A60BD42C20080800A2000530FE2CA20093
:1009E0000230FE2CA2000630FE2CA2000330FE2CAA
:1009F000A2000430FE2CA2000130FE2CA800230827
:100A00002102031D052D22082002043003180130A5
:100A1000031902302805031DFF300800A008031940
:100A2000192D2025A0030000000000000000000098
:100A30000E2DA108031908002025A103A0030E2DE7
:100A40000C30A500A50B222D000000001230A200E2
:100A5000A20B2F2D31253125000000000800312583
:100A6000282D0D30A400A40B332D000008001030F9
:100A7000A8020001031C013EA902031C0800402D2E
:100A80000A30A8020001031C013EA902031C080051
:100A9000402D2A0880042008A8002108A900372535
:100AA0000130A202031CA3032A0980052008A80024
:100AB0002108A9003725A208031D492DA308031DFD
:040AC000492D0800B4
:02400E00C433B9
:00000001FF
